:020000040800F2
:10000000F8160020850100088B0500081D04000873
:1000100089050008F10100089B0E0008000000009F
:10002000000000000000000000000000AB0C000811
:10003000F301000800000000A90500087D0D00087C
:100040009F0100089F0100089F0100089F01000810
:100050009F0100089F0100089F0100089F01000800
:100060009F0100089F0100089F0100089F010008F0
:100070009F0100089F0100089F0100089F010008E0
:100080009F0100089F0100089F0100089F010008D0
:100090009F0100089F0100089F0100089F010008C0
:1000A0009F0100089F0100089F0100089F010008B0
:1000B0009F010008490E00089F0100089F010008E9
:1000C0009F0100089F0100089F0100089F01000890
:1000D0009F0100089F0100089F0100089F01000880
:1000E0009F0100089F0100089F0100080000000018
:1000F0000000000000000000000000000000000000
:1001000000000000000000009F0100089F0100089F
:100110009F0100089F0100089F0100089F0100083F
:100120009F0100089F0100089F0100089F0100082F
:100130009F0100089F0100089F0100089F0100081F
:100140009F0100089F0100089F0100089F0100080F
:10015000DFF80CD000F03AF800480047012400080E
:10016000F8160020EFF30980704780F30988704784
:10017000EFF30880704780F30888704740BA7047F3
:10018000C0BA70470648804706480047FEE7FEE7CA
:10019000FEE7FEE7FEE7FEE7FEE7FEE7FEE7FEE737
:1001A000ED0D000851010008D2B201E000F8012B6A
:1001B000491EFBD270470022F6E710B513460A46E7
:1001C00004461946FFF7F0FF204610BD064C074DC8
:1001D00006E0E06840F0010394E807009847103417
:1001E000AC42F6D3FFF7B8FF342F0008542F0008B5
:1001F000FEE7704701B50098411E00910028FAD132
:1002000008BD00000149C86070470000002002409E
:1002100070B50D4E0546304600F088F8042811D11F
:100220000A4C206940F0020020616561206940F0BD
:1002300040002061304600F079F8216941F6FD72F6
:100240001140216170BD0000FFFF0F00002002403F
:1002500008490420CA68D20701D001207047CA6843
:10026000520701D502207047C968C906FBD5032093
:1002700070470000002002400248016941F08001FF
:100280000161704700200240F0B506464FF6FF7747
:100290000D46384600F04AF804280DD1074C206975
:1002A00040F0010020613580384600F03FF82169B8
:1002B00041F6FE7211402161F0BD000000200240B5
:1002C0002DE9F841064600204FF6FF7700900D46D5
:1002D000384600F02BF8042817D10D4C206940F067
:1002E000010020613580B846384600F01FF841F61D
:1002F000FE77042806D1B61C280C009630804046B4
:1003000000F014F8216939402161BDE8F88100004E
:1003100000200240034802494160034941607047A0
:100320002301674500200240AB89EFCD00B50346AD
:10033000FFF78EFF02E0FFF78BFF5B1E012803D063
:10034000002B00D1052000BD002BF4D1FAE7F0B559
:10035000CC78002204F00F03E40601D58C78234307
:100360000C784FF00F0C4FF0010EDCB105680E88D1
:100370000EFA02F42640A64210D196000CFA06F7B7
:1003800025EA070703FA06F5CE783D43282E02D06A
:10039000482E02D002E0446100E00461521C082AA9
:1003A000E5D305600A88FF2A1CD94468002202F1BF
:1003B00008060EFA06F50E882E40AE420ED19600C3
:1003C0000CFA06F7BC4303FA06F7CE783C43282E16
:1003D00000D14561CE78482E00D10561521C082A13
:1003E000E5D34460F0BD41617047016170470AB1D7
:1003F0000161704741617047064801680648016025
:100400000449091F09684160024908390968816087
:1004100070470000F0F7FF1F80000020FEE700009B
:100420002DE9F047DFF878A0DAF800001D4988428E
:1004300034D10AF104000068A0F52051B1F5BC3FA9
:100440002CD84FEA9008800701D008F10108164E19
:10045000164DFFF75FFF002717E0D6F80090002445
:10046000680502D12846FFF7D3FE49462846FFF724
:1004700027FF042803D0641CE4B2032CF5D32868BA
:10048000814504D1361D2D1D7F1C4745E5D35046BF
:10049000FFF7BEFEBDE8F047FFF7EEBEBDE8F08710
:1004A000005802084433221100600208008000084E
:1004B000F8B501211C2000F079F84FF40076ADF872
:1004C000006010242D4F8DF8034003258DF8025055
:1004D00069463846FFF73BFF31463846FFF785FF50
:1004E0000120ADF800008DF803408DF802506946F8
:1004F0003846FFF72CFF01213846FFF776FF022030
:10050000ADF800008DF803408DF80250694638467A
:10051000FFF71DFF02213846FFF767FF2020ADF8E7
:100520000000174E8DF803408DF8025069463046A2
:10053000FFF70DFF20213046FFF755FF44F207007B
:10054000ADF800008DF803400E4C8DF8025069465E
:100550002046FFF7FCFE01212046FFF744FF022161
:100560002046FFF740FF04212046FFF73CFF4FF4F1
:1005700080412046FFF737FFF8BD0000000801402A
:1005800000100140000C0140FEE770474FF4A060EE
:10059000AFF3008002490843024908607047000039
:1005A0000000FA050CED00E070470000044A002945
:1005B000916901D0014300E08143916170470000DF
:1005C00000100240F0B52B4C61682B4A11F00C0171
:1005D0004FF00F0603D0042901D0082901D0026092
:1005E00026E06168636806EA914103F480330D29CF
:1005F00001D0891C00E00621BBB1E36A13F4803FFF
:10060000E36A03F00F0303F101030AD0E56AC5F3BF
:100610000317E56A7F1CB2FBF7F2C5F30325AD1C97
:100620006A43B2FBF3F24A43D9E7144A51430160EB
:100630006168134A06EA1111535C0168D9404160B0
:100640006368072505EA1323D35C21FA03F383606B
:10065000636805EAD323D25CD140C160626803239A
:1006600003EA9232064B1B1F9A5CB1FBF2F1016167
:10067000F0BD00000010024000127A0000093D00A9
:100680006400002010B5012210210448FFF7AFFEDE
:10069000BDE81040FF2000F09DBA000000080140B6
:1006A00070B5054601220021092000F0CFF90400B1
:1006B00004D11021284600F047F90446FFF7E2FF75
:1006C0000CB1012070BD002070BD70B505464FF61D
:1006D000FF7401E0641EA4B2FF2000F07DF9A8427F
:1006E00002D0002CF6D102E00CB1002070BDFF203A
:1006F00070BD1FB56846FFF7D3FF10B1002004B0EE
:1007000010BD9DF800100120B0EB911F09D19DF89C
:1007100008209DF8091000EB02200844000480091D
:10072000EDE79DF805009DF80A1000F00F0000EBC2
:10073000D1109DF809109DF8072001F0030100EB8E
:1007400041019DF80800800900EB82009DF8062019
:1007500002F0030200EB8220401CC91F8840CEE754
:100760002DE9F84300F00CF9382000F05FFA00F0B2
:1007700035F900204FF47061401C80B28842FBD3F1
:100780000024FF2000F026FA641CA4B20A2CF8D33F
:10079000C82400219522084600F058F90546012892
:1007A00004D02000A4F10104A4B2F2D14A4E0027E3
:1007B000012D377068D187224FF4D571082000F0E1
:1007C00045F94FF6FE78012820D00122002137207C
:1007D00000F03CF901220021292000F037F901281E
:1007E00053D802203070444601220021372000F007
:1007F0002DF901220021292000F028F9050053D00D
:100800002000A4F10104A4B2EED14DE000246F4613
:10081000FF2000F0E1F83855641CA4B2042CF7D393
:100820009DF80200012847D19DF80300AA2843D172
:1008300044464FF0804801220021372000F006F99D
:1008400001224146292000F001F9050004D02000D2
:10085000A4F10104A4B2EED1B4B1012200213A20E6
:1008600000F0F4F880B90024FF2000F0B5F8385506
:10087000641CA4B2042CF7D39DF80000400601D5F7
:10088000062000E00420307016E00120307044465D
:1008900001220021104600F0D9F8050004D0200004
:1008A000A4F10104A4B2F3D12CB101225102102011
:1008B00000F0CCF800B13770FFF7E4FE102000F034
:1008C000B5F9307810B10020BDE8F8830DB12846A5
:1008D000FAE7AA20F8E70000180000202DE9F0410F
:1008E0000646184815460078062800D049024FF4FD
:1008F0000077012D4FF0010219D0122000F0A6F868
:100900003946304600F020F86D1E044606F50076A4
:1009100015F0FF0501D0002CF2D0012200210C209F
:1009200000F094F8FFF7AEFE2046BDE8F0811120FC
:1009300000F08CF80400F5D13946304600F004F898
:100940000446EFE71800002070B504460D46FE206F
:10095000FFF7BBFE28B1012070BD00F03BF904F8A1
:10096000010B2800A5F10105ADB24FF0FF00F4D155
:1009700000F030F9FF2000F02DF9002070BD0000DC
:1009800038B501210420FFF711FE01211020FFF7E7
:100990000DFE1024ADF8004014208DF80300032054
:1009A0000B4D8DF8020069462846FFF7D0FCADF8E4
:1009B000004048218DF8031069460648FFF7C7FC40
:1009C00000F0C4F8012210212846FFF710FD38BDC1
:1009D000000801400010014000F0FCB810B50022F2
:1009E00010210548FFF703FD00F061F8002802D050
:1009F000FFF748FE012010BD0008014070B50C460D
:100A0000054600F054F808B1012070BD204600F002
:100A1000E1F8FD2C18D000244FF40076285D00F09A
:100A2000D9F8641CA4B2B442F8D3FF2000F0D2F885
:100A3000FF2000F0CFF8FF20FFF7CEFF00F01F00EF
:100A4000052801D0022070BD002070BD70B516468B
:100A50000C460546FFF716FEFFF7C0FF08B1FF2062
:100A600070BD45F0400000F0B5F8200E00F0B2F87F
:100A7000C4F3074000F0AEF8C4F3072000F0AAF872
:100A8000E0B200F0A7F8304600F0A4F80C2D02D137
:100A9000FF2000F09FF8FF24FF20FFF79DFF0106D5
:100AA000DED52100A4F10104E4B2F5D170BD10B58A
:100AB0000024FF20FFF790FFFF2804D0641C601C77
:100AC000F7D1012010BD002010BD000070B5064612
:100AD0001D4815460C460078062800D04C02012D12
:100AE00013D0012809D0012200213720FFF7AEFFE3
:100AF000012229461720FFF7A9FF012221461920CC
:100B0000FFF7A4FF04000AD01AE0012221461820B2
:100B1000FFF79CFF040013D1FE2130460DE0FC21BD
:100B20003046FFF76BFF6D1E06F5007615F0FF05EA
:100B300001D00028F3D0FD210020FFF75FFF04461D
:100B4000FFF7A0FD204670BD1800002010B586B04C
:100B500001210520FFF72AFD01210803FFF726FDEB
:100B6000E020ADF8140018208DF8170003208DF850
:100B7000160005A91548FFF7EAFB0020ADF80000B4
:100B80004FF48271ADF80210ADF804000221ADF807
:100B900006100121ADF808104902ADF80A103821FD
:100BA000ADF80C10ADF80E000720094CADF81000A0
:100BB0006946204600F05DF80121204600F044F827
:100BC000FF2000F007F806B010BD0000000801404B
:100BD000003001402DE9F041074600244FF4FA654A
:100BE000114E03E0641CA4B2AC420FD8022130467F
:100BF00000F034F80028F5D03946304600F037F8D8
:100C0000002406E0641CA4B2AC4202D90020BDE876
:100C1000F0810121304600F021F80028F2D0304662
:100C200000F023F8C0B2F2E7003001400146054869
:100C3000028822F03802028002880A4302800121E1
:100C400000F002B8003001400029018802D041F0D4
:100C5000400101E021F04001018070470246002080
:100C600012890A4200D00120704780897047818133
:100C7000704730B502884C8802F441530A88CD8809
:100C800022438C882C4322430C8922434C892243E3
:100C90008C892243CC8922431A430280828B22F41E
:100CA00000628283098A018230BD70470CB500233F
:100CB0002E4800930193016841F4803101604FF6A2
:100CC000FF71026802F400320192009A521C0092F5
:100CD000019A12B9009A8A42F3D10168890342D578
:100CE0000121019122490A6842F010020A600A6853
:100CF00022F003020A600A6842F002020A604168B8
:100D0000416041684160416841F480614160C16A6D
:100D1000184A1140C162C16A174A1143C162016891
:100D200041F08061016001680901FCD5416821F44E
:100D30007C114160416841F4E8114160016841F073
:100D40008071016001688901FCD5416821F00301CF
:100D50004160416841F0020141604168C1F3810195
:100D60000229FAD10CBD01930CBD00000010024015
:100D70000020024000F0FEFF140801000C488168CA
:100D8000491C81604168491C416081684FF47A7256
:100D9000B1FBF2F302FB1311012902D1C168491C16
:100DA000C1600178002901D1012101707047000064
:100DB000500000200B484FF47A710068B0FBF1F04E
:100DC000B0F1807F0DD220F07F414FF0E020491E2E
:100DD0004161054AF0211170002181610721016103
:100DE0007047FEE70400002023ED00E0124810B534
:100DF000016841F0010101604168104A1140416001
:100E000001680F4A11400160016821F480210160EE
:100E1000416821F4FE014160016821F0A0510160A8
:100E20004FF47F0181600021C162FFF73FFF054958
:100E30004FF00060086010BD001002400000FFF09D
:100E4000FFFFF6FE08ED00E010B50A4C0121204638
:100E500000F017F800280AD00121204600F00EF813
:100E60000549D1F8900118B10020C1F8900110BDDA
:100E70000120FAE70004004000002342C943018238
:100E8000704702460020138A92890B4202EA01024F
:100E900002D0002A00D001207047FEE702E008C817
:100EA000121F08C1002AFAD170477047002001E0E4
:100EB00001C1121F002AFBD17047000070B50F4C12
:100EC0008318A34201D9032070BDA2B101250023DC
:100ED0000BE004780E78A64204D0FF2C01D002204B
:100EE00070BD0025401C491C5B1C9342F1D3012DB1
:100EF00001D0012070BD002070BD0000000002087C
:100F00002DE9F0418846074615462649042628441F
:100F1000884202D90120BDE8F081EDB3E80700D096
:100F2000551C2A4641463846FFF7C8FF0400F2D058
:100F3000012080F31088FFF7EDF93520FFF762F903
:100F4000022C06D1F80AC002FFF762F9064604280F
:100F500021D14FF47A700100A0F1010080B2FAD1E2
:100F600000240EE008EB440118F81400497840EA28
:100F700001213846FFF788F90646042804D1BF1C32
:100F8000641CB4EB550FEDD3FFF776F9002080F326
:100F90001088042E03D000E001E00220BBE700200F
:100FA000B9E700000000020810B5044600202071D7
:100FB000401EE062204601F0AAFA08B1032010BDED
:100FC000B4F82E02A0F52A41553901D0022010BDF7
:100FD00094F86600B4F8671040EA01210848B0EBC5
:100FE000012F08D094F88210B4F8832041EA02213E
:100FF000B0EB012F01D1002010BD012010BD000079
:101000000046415400E0401C02780AB18A42FAD1FD
:10101000D0B2704770B5FFF77DF90C4C4020E0600E
:101020003420FFF7EFF80020094DA06007E005EB42
:101030008020FFF7EDF86070A068401CA060E168B8
:10104000884202D261780429F1D070BD18000020D6
:1010500000800008426A0068121D490A8078B1FBCE
:10106000F0F002CA21B1884204D3401A121DF8E7F9
:10107000002070471168084470474269891E921E1B
:101080008A4201D800207047826A807801FB0020E4
:1010900070472DE9F0410F00064606D001F02CF90B
:1010A000022809D20120BDE8F081F56815B1706908
:1010B000A84207D8012505E0411CF4D0716981429E
:1010C000F1D83D462C467069641CA04202D8022427
:1010D000022D0AD32146304601F00EF938B1411CE9
:1010E000E1D00128DFD0AC42EDD10020DBE76FF08A
:1010F00070422146304601F0E9FA30B957B1224634
:101100003946304601F0E2FA20B101280DD0012421
:101110002046C8E7F4603069411CF9D0401E3061B8
:10112000707940F001007071F2E74FF0FF34EFE7A3
:101130002DE9F35F88460D6800E06D1C28782F28A4
:10114000FBD05C28F9D0009800242646D0F81C90EB
:10115000A85D761C202815D32F2813D05C2811D029
:10116000FF2C2FD2012100F0DBFE07002AD0802FB8
:1011700004D201465FA0FFF745FF18BB29F81470A1
:10118000641CE5E7AA19C8F80020202801D204262B
:1011900016E0002614E009EB440030F8020C202889
:1011A0000DD02E280BD06CB1002129F81410009816
:1011B0000B222021806901F0A3F9002706E0641EBC
:1011C000002CE8D10620BDE8FC9F7F1C39F81700F1
:1011D0002028FAD02E28F8D01FB146F0030600E0F0
:1011E000641E2CB109EB440030F8020C2E28F7D114
:1011F0004FF0000AD0464FF0080B39F817507F1C0B
:1012000005B3202D03D02E2D04D1A74202D046F0E5
:101210000306F2E7DA4501D2A74219D1BBF10B0F61
:101220000ED0A74201D046F003060BD84FEA8860E3
:1012300027464FF0080A4FF00B0B4FEA1068DCE727
:1012400046F00306009880690178E5292ED02FE04A
:10125000802D0CD30021284600F062FE050003D04B
:101260002748284410F8805C46F0020625B129463C
:1012700024A0FFF7C7FE18B15F2546F003060EE075
:10128000A5F14100192802D848F0020807E0A5F1AD
:101290006100192803D8203D48F00108ADB200983C
:1012A000816901F80A500AF1010AA6E705210170D7
:1012B000BBF1080F03D14FEA88604FEA1068C8F30A
:1012C0008100032803D06FEA0801890701D146F0A5
:1012D0000206B10709D408F00301012901D146F043
:1012E0001006012801D146F0080600988069C672F0
:1012F000002068E7222A3A3C3E3F7C7F0000000045
:10130000B82900082B2C3B3D5B5D000070B50E46F4
:101310000546002100F087FA88B900242969286869
:1013200001F0F5F858B969690978E5290BD051B190
:1013300000240121284600F0A1F80028EED004285E
:1013400000D1072070BD641CB442F2D170BD000012
:101350002DE9F05F0446002100F065FA00287AD1FB
:10136000FF254FF6FF70AB4620842169206801F00D
:10137000CEF807007CD16669307848B1F17AE5286B
:1013800001F03F0169D00A0704D50F2965D105E0B6
:1013900004276DE00F2901D08DB34DE0E16979B3E9
:1013A000420606D596F80DB020F04000E2880546CA
:1013B0002284A84236D1727B5A4533D130788A468E
:1013C00020F04000401EB14600EB800101EBC0065A
:1013D0004FF000080127284810F8081001EB090019
:1013E000008877B100F0BCFD0746FF2E1AD23AF80C
:1013F0001600761C00F0B4FDB84213D105E016E0EB
:101400002FE0A0F57F41FF390CD108F10108B8F1B8
:101410000D0FE0D399F80000400606D52FB13AF839
:10142000160010B1FF25EDB21BE06D1EFBE7304644
:1014300001F022FA58451BD0A069C17AC9070CD126
:101440000B210022491E07D316F8012B10F8013B8F
:10145000D21AF7D001E00CE052B14FF6FF70FF2531
:1014600020840021204600F009F807003FF47DAFFA
:101470003846BDE8F09F0000382A00082DE9F04109
:10148000C78804467F1C38040E46000C2CD0206907
:1014900050B339075AD1401C2061E168206829B156
:1014A0008278521E12EA171F04D04FE00089B8421A
:1014B0001AD94BE000F020FF0546012819D9681C15
:1014C00030D020684169A9423AD86EB1E168FFF78F
:1014D000E0FD05000BD0012D0BD0681C22D0206848
:1014E00001F02FFAF0B906E00420BDE8F0810720F2
:1014F000FBE70220F9E720684FF40072303000214A
:1015000000F0FEFF29462068FFF7B7FD216800269E
:101510004FF00108C8620CE080F80480206801F0F8
:1015200010FA08B10120E0E72068C16A491C761C66
:10153000C16220688178B142EED8C16A891BC1625C
:10154000E56029462068FFF798FD2061E78007F0F5
:101550000F013022206802EB411108446061002035
:10156000C3E700002DE9F35FFF2504462E4604275C
:101570004FF6FF7A4FF0000B67E0206800F0C7FFDE
:10158000070066D16269107878B1D17AE52801F058
:101590003F0108D02E2806D0082908D00023DDF806
:1015A00004C0634505D0FF2540E0042751E0012336
:1015B000F5E70F2901D0B5BB3FE0410605D5567BC5
:1015C00020F04000E18805462184A8422CD1507BC0
:1015D000B04229D11078DFF8849000F03F00401E1F
:1015E00000EB800101EBC0010020E7690123D44634
:1015F00019F800809044B8F8008033B1FF2913D265
:1016000027F811804346491C01E0E0450CD1401CFD
:101610000D28EDD31078400603D5FF2904D227F812
:1016200011B06D1E01E00DE0FF25EDB20021204656
:10163000FFF724FF070008D00BE0104601F01CF96B
:10164000B04208D0A4F820A005E02169002994D177
:101650000FB1C4F810B03846BDE8FC9F382A000826
:101660002DE9FF5F04460C22D4E906763946684628
:1016700000F03EFF9DF80B00C00718D00020F87264
:101680000125E0612B4632466946384600F0F2FDFE
:101690002046FFF75DFE10B96D1C642DF2D3642D5A
:1016A0000BD004280AD19DF80B00F872E6619DF872
:1016B0000B0080070FD5002004E0072004B0BDE830
:1016C000F09F401C36F810100029FAD119300D2176
:1016D000B0FBF1F500E0012529462046FFF716FE94
:1016E00006006BD16D1E50D0E088411B204600F0F3
:1016F0009AF8060062D1A06901F0BEF84FF6FF7AB1
:1017000003902169206800F002FF060056D161694C
:10171000D4F81C90039848730F20C87200200873F7
:101720008876EEB2C876701E00EB800202EBC00332
:101730000022DFF88CB001F1010801E0504502D031
:1017400039F813005B1C1BF802C001F80C001BF8F1
:1017500002704FEA102C07F808C000B95046521C1E
:101760000D2AEBD3504502D039F8130008B946F0E2
:1017700040060E7021680120087100212046FFF705
:101780007DFE06001AD16D1EBBD12169206800F0D4
:10179000BEFE060012D120220021606900F0B0FEDA
:1017A000D4E905010B2200F0A3FEA0696169C07AAB
:1017B00000F01800087321680120087130467DE7A9
:1017C000382A00082DE9F041018C0446C688A1F5AD
:1017D0007F40FF3800D13146204600F024F8050054
:1017E0001ED1E5274FF001082169206800F08FFE27
:1017F000050012D120220021606900F081FE60699D
:101800000770216881F80480E088B04208D2002186
:101810002046FFF733FE0500E6D0042D00D1022557
:101820002846BDE8F08170B5C18083680D46044646
:10183000012B34D020684169994230D923B901780D
:10184000032904D1436A13B18078060110E00189AD
:10185000A94224D9406A11E000F04EFD0346401C25
:101860001BD0022B1BD320684069984217D9AD1BAF
:101870002068B5421946EFD2FFF7FFFBE36070B175
:1018800000EB1510206105F00F013022206802EBFB
:10189000411108446061002070BD012070BD02202C
:1018A00070BD10B530B9FEF75BFF002803D0FF20F4
:1018B000FFF792F8012010BD10B5144660B939B198
:1018C000012912D0022909D003290AD0042010BD11
:1018D000FFF7EDF80028FAD0012010BD4FF400709A
:1018E00000E008201080002010BDFEF702FF2060FD
:1018F000F9E770B514460D460BB160B901E004205C
:1019000070BDDAB221462846FEF7E8FF0028F7D07E
:10191000FF20FFF761F8012070BD0020704770B50F
:1019200014460D460BB148B901E0042070BDDAB28F
:1019300021462846FFF7CAF80028F7D0012070BDDD
:1019400010B5044600F080F9002806D1204601F0C9
:1019500020F8002801D10021216010BD17B581B009
:10196000144602980090684600F023FD002802DA31
:101970000B2004B010BD0B4B002253F8201001B116
:101980000A700199002900D00A7043F8201001D094
:10199000012C01D00020ECE7002202A901A800F0F0
:1019A000F1FAE6E7EC0C00202DE9F74F8CB00600C9
:1019B0000ED04FF0000902F01F0727F001020DA919
:1019C0006846C6F8009000F0DDFA040004D095E007
:1019D00009200FB0BDE8F08F4FF4007000F0BCFAA2
:1019E0005FEA00080AD009A8CDE9060868460D9903
:1019F00000F0E4FB059D040002D003E01120E8E7BD
:101A000005B9062417F01C0F4CD054B1042C03D197
:101A10006846FFF725FE0446059D47F0080754B1C8
:101A200052E0E87A10F0110F01D007244CE078075B
:101A300001D5082448E0380742D500F0B8FCA87367
:101A4000010AE973010C2974000E687485F80B9083
:101A500085F81C9085F81D9085F81E9085F81F90DC
:101A60002946009800F0C3FC82460021284600F079
:101A7000FBFE00990120BAF1000F08711ED00098FA
:101A80005146D0F82CB000F09DFE04001CD1009906
:101A9000AAF10100C8605946009800F038FD040022
:101AA0000AD011E084B9E87AC10601D504240BE01C
:101AB000B90701D5C007B8D1380701D547F02007CD
:101AC0000098C06AC6E90705404600F047FAACB97D
:101AD000B77186F807904F462946009800F087FCBA
:101AE0003061287FD5F81D1040EA0120C6E9027058
:101AF000B761776200983060C088B080204668E7A0
:101B00002DE9F84F894600219A4616460446196089
:101B100000F03FFF002812D1E07900280FD1A07912
:101B2000C0070BD0D4E90210401A04F128014FF08D
:101B3000010B0091864200D9064680E00720BDE8EF
:101B4000F88FA168C80562D120688278521E02EA27
:101B5000512212F0FF0510D129B1626A2AB1204644
:101B6000FFF778FA04E0206902E0616900F0C4FB45
:101B7000022819D3411C44D0606161692068FFF7D5
:101B80007CFA88B100EB0508770A21D02068EA19B1
:101B900081788A4200D94F1B40783B4642464946ED
:101BA000FFF7A7FE68BB02E00220E071C7E7A0795B
:101BB00040060BD5A169A1EB0800B84206D209EB9B
:101BC00040204FF40072009900F092FC7D022CE05E
:101BD000A269424519D0A07940060AD520680123A0
:101BE00000994078FFF79BFE58B9A07920F040009B
:101BF000A07120680123424640780099FFF779FEE2
:101C000018B184F807B0012099E7C4F8188020893A
:101C1000C0F30800C0F50075B54200D9354601197A
:101C200028312A46484600F063FCA068A9442844AD
:101C3000A060DAF800004119761BCAF80010002EE7
:101C40007FF47FAF00207AE770B5044600F0A1FE74
:101C500000280ED1A1798A060BD548060ED520683A
:101C6000012304F128014078A269FFF758FE08B16A
:101C7000012070BDA07920F04000A071E1692068CA
:101C800000F045FC0028F4D1256AE87A40F02000F5
:101C9000E872207B2877A089000A6877E068000C4A
:101CA000A877E068000EE8772846216900F0DCFD9F
:101CB00000F07DFBA875010AE975010C2976000E7C
:101CC00068760020A874E874A07920F02000A07144
:101CD0002168012008712068BDE8704000F0D9BD7E
:101CE000F1B596B0012216A9684600F04BF9040040
:101CF00053D14FF4007000F02FF9070009D012A85B
:101D0000CDE906076846169900F058FA040003D09A
:101D100040E0112017B0F0BD059E56B1F07AC00723
:101D200000D007243146009800F061FB054614B14D
:101D300030E00624F6E7F07AC0061BD5022D01D26A
:101D4000022427E02422694609A800F0D1FB0221E1
:101D500009A80B95FFF767FD04001BD1002109A816
:101D6000FFF700FC040003D0042C03D014B111E0F1
:101D700007240FE06846FFF725FD04000AD12DB1C6
:101D80002946009800F01EFD040003D1009800F0E1
:101D900080FD0446384600F0E1F82046BAE72DE918
:101DA000F84F894600219A4616460446196000F00D
:101DB000F0FD002806D1E079002803D1A079800742
:101DC00002D40720BDE8F88FA06804F12801821929
:101DD0004FF0010B0091824273D392E0A168C805D5
:101DE00073D122689078401E00EA512010F0FF0560
:101DF00018D129B1606A38B12046FFF72BF907E006
:101E0000206938B9002100E061691046FFF741F907
:101E1000002879D001282BD0411C4ED06061216967
:101E200001B92061A07940060BD520680123A26981
:101E300040780099FFF773FD78BBA07920F040004F
:101E4000A07161692068FFF718F988B100EB0508F7
:101E5000770A23D02068EA1981788A4200D94F1B7B
:101E600040783B4642464946FFF759FDA8B902E093
:101E70000220E071A6E7A169A1EB0800B8420AD2EE
:101E800009EB40214FF40072009800F031FBA0797B
:101E900020F04000A0717D0229E00EE0A1694145DB
:101EA00011D0D4E9020188420DD2206801234246B4
:101EB00040780099FFF71DFD28B184F807B0012094
:101EC00080E721E001E0C4F818802089C0F3080011
:101ED000C0F50075B54200D93546204428302A4661
:101EE000494600F005FBA07940F04000A071A068D1
:101EF000A9442844A060DAF800004119761BCAF80A
:101F00000010002E7FF46AAFD4E90201884200D9A4
:101F1000E060A07940F02000A071002052E70000AE
:101F2000802804D30B4A49B1FF2801D9002070470B
:101F300002EB4000A0F580700088704732F8113045
:101F4000834203D0491C89B28029F7D38031C8B2BB
:101F500070470000722A000800F094BA00F062B9DD
:101F60000021064B00E0491C33F81120002A04D060
:101F70008242F8D1024830F811007047722B0008F5
:101F8000522D00082DE9FF474FF000090746C0F821
:101F900000901646084600F00CFA051E03DA0B20E6
:101FA00004B0BDE8F087814850F825408CB13C6012
:101FB000207820B16078FFF7B0FCC1070BD084F81F
:101FC0000090E8B26070FFF76CFCC10708D00320F6
:101FD000E6E70C20E4E70EB1400704D40020DFE779
:101FE0001EB1400701D50A20DAE700252946204620
:101FF000FEF7DAFF012821D100206E4604EB001124
:1020000001F5F7710A792AB10A7AD1F8091042EA82
:10201000012100E0002146F82010401C0428EDD3E7
:10202000002756F8275025B129462046FEF7BCFF69
:1020300000E0022040B17F1C042FF2D3032801D01E
:10204000F0BB01E00120ABE7B4F83B00B0F5007F46
:102050005DD1B4F8461029B994F85400D4F855105D
:1020600040EA0121A16194F840C084F803C0BCF1AA
:10207000010F02D0BCF1020F49D194F83D600CFB76
:1020800001FCA670E6B1701E064240D1B4F84120B2
:10209000228110073BD1B4F8430028B994F85000CE
:1020A000D4F8513040EA0320E38F4BB103EB0C0727
:1020B00007EB1217B8422AD3C01BB0FBF6F000E0C2
:1020C00025E020B3012640F6F678404500D30226ED
:1020D0004FF6F678404500D30326801C2F44A762B4
:1020E0002B446061C4E90753032E12D07AB103EB8D
:1020F0000C026262022E17D000F0010200EB4000D9
:1021000002EB500000F2FF10B1EB502F0ED20D2069
:1021100046E7002AFBD194F85C20D4F85D308000BB
:1021200042EA03226262EDE74000EBE74FF0FF3046
:102130002061E06080206071032E30D1B4F860002F
:1021400001282CD1691C204600F0E1F938BB84F845
:102150000590B4F82E02A0F52A4155391FD194F804
:102160003000D4F8311040EA01201149884216D1DC
:1021700094F81402D4F8151240EA01200D4988425F
:102180000DD194F81802D4F8191240EA0120206108
:1021900094F81C02D4F81D1240EA0120E0600649C0
:1021A00026700888401C0880E08017E7EC0C0020AF
:1021B00052526141727241617400002073B504464D
:1021C000019908782F2801D05C2801D1491C019180
:1021D0000025A56001980078202805D2002120461E
:1021E000FFF721FB65617CBD01A92046FEF7A0FF3A
:1021F0000028F8D12046FFF7ABF8A169C97A28B1C9
:102200000428F0D14907EED405207CBD4907FCD451
:102210006169C87AC006F7D5206800F0E8F8A060C8
:10222000E2E7000010B5002821D0114B001F00226A
:10223000196803E0814203D80A4649680029F9D1A8
:1022400052B11368841A9C4204D10068184410608B
:10225000104602E0506000E0186039B102680B1AC5
:10226000934203D10B681A4402604968416010BD73
:10227000780000207CB516461C4605460B2200F06F
:1022800037F9052C14D91B4A0FE006F102064FF06E
:1022900000012346044663F35F044FEA5000E30362
:1022A00000D55440491C1029F3D330880028ECD1C4
:1022B00007216B4604F00F003030392800D9C01DCB
:1022C0005854491E2409F5D17E205854002200E0BC
:1022D000521C8A4202D2A85C2028F9D1082902D2D5
:1022E000585C491C00E02020A854521C082AF5D351
:1022F0007CBD0000211001002DE9F0410D4604468F
:10230000022909D36069A84206D92078012806D09D
:10231000022828D0032832D00120BDE8F081206AAD
:1023200005EB550600EB5621204600F0F0F868BB9F
:10233000C6F308002044761C90F83070206A00EB49
:102340005621204600F0E3F800BBC6F30800204405
:10235000E90790F8300047EA002001D00009DCE7E7
:10236000C0F30B00D9E7206A00EB1521204600F0EE
:10237000CEF858B9E8B204EB4000008ECDE7206AF1
:1023800000EBD511204600F0C2F810B14FF0FF303D
:10239000C3E740F2FF1000EA8500204490F83010B7
:1023A000D0F8310041EA002020F07040B5E700206D
:1023B000704710B503464FF0FF301C68002C13D057
:1023C000214600E0491C0A78202A0ED33A2AF9D186
:1023D00014F8012B303A0A2A06D28C4204D1032A7F
:1023E00002D2491C1046196010BD002010BD0246E3
:1023F000488B1278032A02D1898A40EA014070474B
:1024000086B0FEF7F3FCFEF7D5FC6846FEF7DAF877
:10241000FEF7BCF8FDF7F0FF0A20FDF7EBFEFEF734
:1024200047F84FF004084FF00209124D4FF0030A2D
:10243000114E124F124CFDF7F3FF2878012808D0F7
:102440007068386020603068FDF795FE206880472E
:10245000F1E785F8008000F071F810B185F800A070
:10246000E9E7C820FDF7C6FE85F8009000F0DCF92A
:10247000E1E7000000000020008000084800002084
:1024800044000020F0B50B30154D20F0070100246A
:10249000144A0FE003688B420BD38B4205D95E1AB6
:1024A00043184768C3E9006700E04368136002C04F
:1024B00004E0021D10680028ECD12046002802D15B
:1024C000286808B10020F0BD064A07481060074A96
:1024D000121A22F00702C0E9002401202860D7E781
:1024E0007C00002078000020FC0C0020F80E00206A
:1024F00003E011F8013B00F8013B521EF9D270478E
:10250000C9B201E000F8011B521EFBD2704770B542
:102510000446C06A0D46A8420ED0204600F011FACB
:1025200038B9607801232A4604F13001FFF7E1F958
:1025300008B1012070BDE562002070BD2DE9F041B9
:102540004E4DADF58A6D002401224DA14D486C61C0
:10255000FFF704FA06460520FDF74CFE01224AA1CA
:102560006846FFF721FAE87001224AA16846FFF7A2
:102570001BFAE87001224AA16846FFF715FAE870D5
:1025800030004FF0FF3605D06846FFF7D9F9012239
:1025900046A10FE00520FDF72DFE0398A8610B2250
:1025A00043A18AA8FFF700FA60B18AA8FFF7C8F92B
:1025B000012242A10020FFF7D1F930460DF58A6DC6
:1025C000BDE8F081FEF726FDAC804FF40047DFF850
:1025D000F0803C4C3E11A87840B10020A870002843
:1025E0003946404604D0FDF7FEFE03E00120F5E742
:1025F000FDF7FBFEA888314604EBC0202861324875
:10260000FDF7D9FD1D4B324614332F496846FFF7BD
:1026100077FA00BB6A69F2B1B24205D2A8882A49AA
:1026200004EBC020FEF76CFC144B27491C338AA82E
:102630006A69FFF7B4FB8AA8FFF706FB6A69B24232
:1026400005D1A888204904EBC020FEF759FCA888D2
:10265000401CA880BFE78AA8FFF772F96846FFF719
:102660006FF9012211A10020FFF778F9012213A1CF
:102670000020FFF773F90020A0E7000018000020F9
:10268000303A00008C000020303A2F4170702E62EA
:10269000696E0000303A2F546573742E747874009C
:1026A000303A2F546573742E62696E00303A2F00F1
:1026B000303A2F746573742E62696E00313A2F00C0
:1026C0000008014000800008EC0400202DE9F047DC
:1026D00016460D460446022902D36069A84202D874
:1026E0000220BDE8F087207806F0FF084FF00109CE
:1026F000012807D0022837D0032846D0022084F8CA
:102700000490EEE7206A05EB550700EB57212046C1
:10271000FFF7FDFE0028F2D1C7F308002044303057
:10272000E90703D0017868F31F1100E0314601701A
:1027300084F80490206A7F1C00EB57212046FFF7A5
:10274000E6FE0028DBD1C7F3080121443031EA0757
:1027500002D0C6F3071205E00A78C6F3032302F09D
:10276000F0021A430A70CAE7206A00EB15212046DE
:10277000FFF7CDFE0028C2D1E9B204EB4101320AD5
:1027800081F8308081F83120B9E7206A00EBD5115B
:102790002046FFF7BCFE0028B1D140F2FF1101EA4C
:1027A0008501214430314FF07043D1F8012003EA14
:1027B000022232430A70130A4B70130C8B70120EF4
:1027C000CA709CE72DE9F0410F460446022916D352
:1027D0006069B84213D900261FE039462046FFF74A
:1027E0008BFD05001CD0012D09D0681C09D00022EA
:1027F00039462046FFF76AFF060011D103E00226A2
:102800000EE001260CE02069411C05D0401C20612F
:10281000607940F0010060712F466069B842DCD8F1
:102820003046BDE8F081000010B5012206A107483E
:10283000FFF794F806A0FFF753FA0122BDE8104015
:1028400008A10020FFF78AB8303A00008C00002071
:10285000303A2F55706C6F6164436F6E6669672EF6
:1028600074787400303A2F0081760A0AC2760A0C16
:102870000275090E41757047014600200B2243087E
:1028800003EBC01011F8013B521E1844C0B2F6D140
:10289000704770B5044600F054F805004FD1207819
:1028A000032845D16079012842D1420204F1300069
:1028B00000210646FFF724FE552084F82E02AA20A8
:1028C00084F82F02522084F8300084F8310061220D
:1028D00084F83220412084F83300722184F81412E5
:1028E00084F8151284F8160284F81722206984F8F7
:1028F0001802010A84F81912010C84F81A12000E49
:1029000084F81B02E06884F81C02010A84F81D1296
:10291000010C84F81E12000E84F81F02E2690123E4
:10292000521CE26260783146FEF7F9FF00206071C8
:10293000002260781146FEF7BFFF00B1012528464E
:1029400070BD2DE9F0410446007900B3E66A04F158
:1029500030016078012332460F46FEF7E0FF10B1E8
:102960000120BDE8F08100202071206AA169301AA1
:1029700088420CD2E57808E0A0690123064460781B
:1029800032463946FEF7CBFF6D1E022DF4D20020F1
:10299000E7E710B538B1016829B10A781AB1CA88D9
:1029A0008088824201D0092010BD4878FEF7B5FF2B
:1029B000C007F9D0032010BD809A90418E418F80CE
:1029C0004545454949498E8F9092924F994F5555AB
:1029D00059999A9B9C9D9E9F41494F55A5A5A6A795
:1029E000A8A9AAABAC21AEAFB0B1B2B3B4B5B6B77B
:1029F000B8B9BABBBCBDBEBFC0C1C2C3C4C5C6C7DF
:102A0000C8C9CACBCCCDCECFD0D1D2D3D4D5D6D7CE
:102A1000D8D9DADBDCDDDEDFE0E1E2E3E4E5E6E7BE
:102A2000E8E9EAEBECEDEEEFF0F1F2F3F4F5F6F7AE
:102A3000F8F9FAFBFCFDFEFF01030507090E101271
:102A40001416181C1E000004000200018000400043
:102A50002000100008000400020000000080004078
:102A600000200010000800400020001000080004B2
:102A70000002C700FC00E900E200E400E000E5001D
:102A8000E700EA00EB00E800EF00EE00EC00C40015
:102A9000C500C900E600C600F400F600F200FB0025
:102AA000F900FF00D600DC00A200A300A500A720CB
:102AB0009201E100ED00F300FA00F100D100AA005C
:102AC000BA00BF001023AC00BD00BC00A100AB00E9
:102AD000BB00912592259325022524256125622599
:102AE000562555256325512557255D255C255B25F4
:102AF0001025142534252C251C2500253C255E2574
:102B00005F255A25542569256625602550256C25A5
:102B1000672568256425652559255825522553259F
:102B20006B256A2518250C25882584258C2590255C
:102B30008025B103DF009303C003A303C303B500E3
:102B4000C403A6039803A903B4031E22C603B50356
:102B500029226122B1006522642220232123F7006B
:102B60004822B0001922B7001A227F20B200A02507
:102B7000A0006100620063006400650066006700F9
:102B8000680069006A006B006C006D006E006F00E9
:102B90007000710072007300740075007600770099
:102BA000780079007A00A100A200A300A500AC0083
:102BB000AF00E000E100E200E300E400E500E60031
:102BC000E700E800E900EA00EB00EC00ED00EE00B1
:102BD000EF00F000F100F200F300F400F500F60061
:102BE000F800F900FA00FB00FC00FD00FE00FF0009
:102BF000010103010501070109010B010D010F018D
:102C0000110113011501170119011B011D011F01FC
:102C1000210123012501270129012B012D012F016C
:102C200031013301350137013A013C013E014001D8
:102C300042014401460148014B014D014F01510140
:102C400053015501570159015B015D015F016101AC
:102C500063016501670169016B016D016F0171011C
:102C60007301750177017A017C017E019201B10344
:102C7000B203B303B403B503B603B703B803B90390
:102C8000BA03BB03BC03BD03BE03BF03C003C10340
:102C9000C303C403C503C603C703C803C903CA03E8
:102CA0003004310432043304340435043604370468
:102CB000380439043A043B043C043D043E043F0418
:102CC00040044104420443044404450446044704C8
:102CD000480449044A044B044C044D044E044F0478
:102CE0005104520453045404550456045704580420
:102CF00059045A045B045C045E045F047021712172
:102D0000722173217421752176217721782179210F
:102D10007A217B217C217D217E217F2141FF42FF81
:102D200043FF44FF45FF46FF47FF48FF49FF4AFF77
:102D30004BFF4CFF4DFF4EFF4FFF50FF51FF52FF27
:102D400053FF54FF55FF56FF57FF58FF59FF5AFFD7
:102D50000000410042004300440045004600470097
:102D6000480049004A004B004C004D004E004F0007
:102D700050005100520053005400550056005700B7
:102D8000580059005A002100E0FFE1FFE5FFE2FF93
:102D9000E3FFC000C100C200C300C400C500C600FC
:102DA000C700C800C900CA00CB00CC00CD00CE00CF
:102DB000CF00D000D100D200D300D400D500D6007F
:102DC000D800D900DA00DB00DC00DD00DE0078018D
:102DD000000102010401060108010A010C010E01B3
:102DE000100112011401160118011A011C011E0123
:102DF000200122012401260128012A012C012E0193
:102E0000300132013401360139013B013D013F01FE
:102E100041014301450147014A014C014E01500166
:102E200052015401560158015A015C015E016001D2
:102E300062016401660168016A016C016E01700142
:102E400072017401760179017B017D019101910389
:102E500092039303940395039603970398039903AE
:102E60009A039B039C039D039E039F03A003A1035E
:102E7000A303A403A503A603A703A803A903AA0306
:102E80001004110412041304140415041604170486
:102E9000180419041A041B041C041D041E041F0436
:102EA00020042104220423042404250426042704E6
:102EB000280429042A042B042C042D042E042F0496
:102EC00001040204030404040504060407040804BE
:102ED00009040A040B040C040E040F046021612190
:102EE00062216321642165216621672168216921AE
:102EF0006A216B216C216D216E216F2121FF22FF40
:102F000023FF24FF25FF26FF27FF28FF29FF2AFF95
:102F10002BFF2CFF2DFF2EFF2FFF30FF31FF32FF45
:102F200033FF34FF35FF36FF37FF38FF39FF3AFFF5
:102F300000000000542F0008000000208000000066
:102F40009C0E0008D42F0008800000207816000096
:102F5000AC0E00080000000000A24A0400000000BF
:102F60000000000001020304060708090004000035
:102F70000000000000000000000000000000000051
:102F80000000000000000000000000000000000041
:102F90000000000000000000000000000000000031
:102FA0000000000000000000000000000000000021
:102FB00000000000020406080000000001020304F3
:102FC00001020304060708090000000000000000D9
:042FD00000000000FD
:04000005080001519D
